:020000040000FA
:020000007C285A
:040002000034003492
:08000800692EC70000300A2830
:10001000C7004030C80043207C304C2048084C20AA
:1000200047084C204820152008000A30C200182834
:10003000C20B1728080028305526383005203930E3
:1000400005201430052070300520563005206C3016
:100050000520C8305526383005200C3005200130E9
:10006000052001305526482608003F20C60A0319FE
:10007000C50A003E03193E28082035280800450817
:100080008A00460882000E148E148E100E1008008E
:100090000E148E108E140800C9000830CA008E108D
:1000A000C91B8E140E140E10C90DCA0B4F28210047
:1000B0008E1420000E1400000E1021008E1020005F
:1000C00008000830CA0021008E1420000E1403100E
:1000D0008E180314C90D0E10CA0B662821008E104D
:1000E0002000490808008E100E140E108E1408000F
:1000F0008E140E140E10080083018B012100703045
:10010000990020008C018E0122008C018E012300B9
:1001100004308C008E0121003F308C0030308E0086
:10012000240033308C0030308E00270033309200B2
:10013000220082309700210008309D0093309E00FD
:1001400008309500200095018B128B118B170E1132
:100150008E140E1452261B200C3005203221333011
:100160000C05213A0319D2288E150230BA008030CE
:1001700005208030C500F330C6003520C030052092
:10018000352063266326803005203520C0300520C9
:10019000352063266326BA0BB7288E11013005205F
:1001A00063266326A901A917AA01B301B40133305C
:1001B0000C05123A0319EC2D0E0E0339033AA30075
:1001C000031DE4280530EF28023023020318EA2833
:1001D0000930EF28031DEE280630EF281630A8005E
:1001E000B821CE21322A46346D3453347434653408
:1001F000723465346F340034523461346434693499
:100200006F344934493449340034563465347234D7
:10021000203431342E3431343234003420346234DA
:10022000793420344D342E34593420340034203481
:1002300056346F346C343A34203420342034003453
:1002400020344C34653476343A342034203420342D
:1002500000342A3420345334653465346B3420340C
:100260002A34003421001D142000452621009D144D
:100270009D18382911131D101B35F1001C0DF000BD
:1002800020007008B6007108B700B8010530B90049
:10029000A9263C08B600F0003D08B700F100B801FF
:1002A0007830B900A426663084008130850015308E
:1002B000BA00003F3702031862290231BA0B5929EC
:1002C0003C306329013FB50090210800C8341C343C
:1002D000C3341D34BE341E34B9341F34B434203416
:1002E000AF342134AA342334A5342534A034273440
:1002F0009B34283496342A3491342B348C342C3467
:1003000087342D3482342E347D3430347834323492
:10031000733434346E3435346934373464343934B6
:100320003930052035080F3970380520350E03396E
:1003300054380520383005200800C03005207008EA
:10034000B6007108B700E7263D0808202E300820C7
:100350003E0808203F08082056300820203008209A
:100360003508C0000D273C0808203D08082008007B
:100370002300A1308600013087000C30A0008030BF
:1003800091009F309200151315140000000013080F
:100390001E00910AA00BC329200008002308230790
:1003A0002307A13E860087010130873D403FA4001E
:1003B000413FA500423FA60003302302031DE5296B
:1003C00002302505A700C030A50508008B132300C7
:1003D000803091009F309200151315161515553079
:1003E0009600AA3096009514000000001511200018
:1003F0008B1708008B132300A13086000130870083
:100400000C30A000803091009F309200151315151C
:10041000951616009300A00B0E2A172A5530960049
:10042000AA309600951400000000910A092A95123E
:1004300055309600AA309600951400000000151162
:1004400020008B170800230823072307A13E8600FE
:1004500087010130873D2408C03F2508C13F260899
:10046000C23F0800A91B3B2AAA1C482A0E111B20C8
:100470000C300520AA10E822A91BF72432219D2167
:10048000A90129170C083339333A031D422A5A2A85
:100490008C1C90220C1CA3222918542A8C1EB622D4
:1004A0000C1EC222A91C652AE822F72432219D21B4
:1004B000A9014E268B123C30A2003830950027301F
:1004C000A0001030A1008B16322A2A1C6A2AD022E2
:1004D0002A10322A291D6F2A32252911322AA91DF4
:1004E0007E2A33187B2A2B08C5002C08C600C03092
:1004F000052035207C2AA125A911322A291E852A0A
:100500002322E621FA212912322AA91E322A0E15A7
:100510008E112700930120008B156300AA14322A44
:100520004E268C18A02A291403302302031D9A2A70
:10053000A710A02AA403240A031DA02A2808A400A7
:100540008C1CA02A08004E260C18B32A291403304C
:100550002302031DAD2AA714B32AA40A24082802E3
:100560000318B32AA4010C1CB32A08004E268C1AC7
:10057000BF2AA914A603260A031DBF2AA6018C1EA2
:10058000BF2A08004E260C1ACD2AA914A60A26084E
:100590000F3C0318CD2A0F30A6000C1ECD2A0800F0
:1005A000C03005208130C5001730C60035200A3024
:1005B00026020318DF2AC63005202608E52AC530A2
:1005C0000520313008200A30260230380820080083
:1005D0002308031DF02A8330C5002B30C600FF2AF4
:1005E000023023020318F92A8330C500A330C60065
:1005F000FF2A031D232B8430C5006B30C60024085E
:10060000C0000310C00DC00D4008C100C00D400D5A
:100610000318C50A41070318C50AC6070318C50A07
:100620008030052035204508AB004608AC00093075
:10063000C6070318C50A3F20AD00C60A0319C50A3C
:100640003F20AE002A2B803005208130C5002930A4
:10065000C600352008004D34493444342D34463426
:100660004D342034203400342034373436342E34A2
:1006700031344D3448347A340034003458345A34E8
:10068000493450342D3446344D3420342034003431
:100690002034373437342E3438344D3448347A34B7
:1006A00000340434983446344D34203441344934D1
:1006B00043344834493400342034383430342E3410
:1006C00037344D3448347A3400340B34D8344E3413
:1006D00048344B34203446344D34203420340034F4
:1006E0002034383432342E3435344D3448347A346E
:1006F00000341034583454344F344B34413449347A
:1007000020342034203400342034393432342E3430
:1007100039344D3448347A3400342A34583443342C
:100720004234433420342034203420342034003404
:100730002034393433342E3437344D3448347A3419
:1007400000342C3458344E34413443344B34353433
:1007500020342034203400342034373439342E34DB
:1007600035344D3448347A3400340834D834543471
:100770004F344B3459344F34203446344D340034E4
:100780002034383430342E3430344D3448347A34D4
:1007900000340A3418344A342D3457344134563432
:1007A00045342034203400342034383431342E346D
:1007B00033344D3448347A3400340D3458344E34A4
:1007C00048344B34203459344B34483420340034CA
:1007D0002034383431342E3439344D3448347A347A
:1007E00000340E34D8344E3448344B34203454342E
:1007F0004B344F34203400342034383432342E34E7
:1008000035344D3448347A34003410345834593443
:100810004F344B344F34483441344D344134003438
:100820002034383434342E3437344D3448347A3428
:1008300000341534D83449346E3474346534723429
:1008400046344D34203400342034383439342E3496
:1008500037344D3448347A340034223458345434E4
:1008600042345334203446344D3420342034003460
:100870002034393430342E3435344D3448347A34DD
:10088000003424345834423455344E344B344134DB
:10089000203446344D3400342034393431342E344D
:1008A00036344D3448347A340034273418344E34D6
:1008B0004934503450344F344E34203420340034D2
:1008C0002034393433342E3430344D3448347A348F
:1008D00000342A34983443344F342E3443344F3464
:1008E0002E344C344F3400342034373436342E34E4
:1008F00035344D3448347A34003401345834423479
:1009000065344834613470347034793421340034BF
:100910002034373438342E3439344D3448347A3432
:1009200000340734583446344D3420344F34533473
:1009300041344B34413400342034383435342E348F
:1009400031344D3448347A3400341634D8344E348B
:1009500048344B34203446344D3420342034003471
:100960002034383438342E3431344D3448347A34E9
:1009700000341E3458344D3442345334203420343F
:1009800020342034203400342034393430342E34B0
:1009900036344D3448347A340034243498344F3467
:1009A0004234433420342034203420342034003482
:1009B0002034393431342E3439344D3448347A3497
:1009C00000342734D8344134423443342034203482
:1009D00020342034203400342034393433342E345D
:1009E00033344D3448347A3400342B345834A91F0E
:1009F000192D432020304C20D0304C2001304C2089
:100A0000033023020319092D2D084C202E084C20F9
:100A10000E2D24084C20250818384C2000304C207E
:100A200000304C2088304C20260880384C2048204C
:100A3000312D291C2A2D033023020319222D0330C6
:100A4000CB25312DD1302704AD000130AE0002306E
:100A5000CB25312D8830AD0026088038AE0005301A
:100A6000CB250800003085002F3084000A30DB25BC
:100A70002F1F322D0B30DB258E112F198E15310CC7
:100A80007F39C0000D27C03005208130C5002030DF
:100A9000C6003520C5300520003085003C3084007C
:100AA0000230BA0012000820BA0B522D0330230284
:100AB00003195B2508002F08C1003008C000C10CD5
:100AC000C00CC10CC00CC10CC030C1058330C500C6
:100AD0002B30C6002808BA004508AB004608AC0019
:100AE0001230C6070318C50A3F20C60A0319C50AF3
:100AF0004002031D802D3F20C039410203198F2D74
:100B0000C60A0319C50ABA0B6C2D803005200830BF
:100B1000BA003F300820BA0B892D33149B2D2B08C7
:100B2000C5002C08C6008030052035204508AB00E4
:100B30004608AC0033104008A40041082704A50073
:100B400008003418A92D2F080339B6003008B70063
:100B5000AD2D2408B6002508B7000230B800F830E3
:100B6000B9009F26E726C0303418803005200030B9
:100B700085003C3084000430BA003A032E3003195B
:100B8000082012000820BA0BBD2D8330C500393073
:100B9000C60035200800C000003085002D308400DC
:100BA000432022304C2040084C2012004C201200E0
:100BB0004C2048200800C000432022304C20400830
:100BC0004C20432023304C20612073201A006120E8
:100BD00078201A004820080033300C063339031DF2
:100BE000EC2D3414A401A501A301AD011830AE0011
:100BF0000230A600F72463266326A12532258C1E29
:100C0000FC2D8C1C1B260C1C2E26291CFF2D2408B9
:100C1000C1002508C000C10CC00CC10CC00CC10C27
:100C2000C030C1054008AD0041081838AE0003309F
:100C3000CB252910FC2D4E268C189A2A2914A503A1
:100C4000250A031D2B2EA403240A031D2B2E01307D
:100C5000A4004030A5008C1C2B2E08004E260C183A
:100C6000422E29140130240203183B2EA50A031D2D
:100C7000422EA40A422EA50A41302502031C422E10
:100C8000A401A5010C1C422E080007300000492ECB
:100C90002730C2004B2EC20B4A2E08001E30552EA4
:100CA0006430552EC830552E0130C300DD30C200EF
:100CB000592E5A2E5B2EC20B582E00005F2E602E2E
:100CC000C30B562E08000A30C4005026C40B652EF4
:100CD000080020000B196F2E0B189A2E9E2E0B1158
:100CE000383095000130A10203197A2E03189E2E88
:100CF000A0029E2EA008031D9E2E2730A0001030BB
:100D0000A1003B30220203192A14393022020319B0
:100D10002915373022020319A91535302202031D87
:100D2000952E291F2916291B2913A20B9E2EA916C1
:100D30008B129E2E2700930120008B110900390889
:100D4000B7073808B63D08003908B7023808B63B7F
:100D500008001030BA003908BF003808BE00BF0DC7
:100D6000BE0D0318B72EBA0BAF2E0314E62EBD012D
:100D7000BC01BF01BE011030BB003A08BB02B73551
:100D8000B60DBF0DBE0DBA0BBF2E38083E02031CB8
:100D9000D92E3E083802031CD12E39083F02031C0D
:100DA000D92E3908BF02031CBE033808BE02031443
:100DB000DA2E0310BD0DBC0DBB080319E52EBB03D5
:100DC000B735B60DBF0DBE0DC52E0310080000309F
:100DD000850040308400FB26FB26FB26FB26FB26F5
:100DE0000430BA00003F303C031DFA2E20301A00B8
:100DF000BA0BF22E08001030BA00C101B735B60D9B
:100E0000C10DF63041070318C1000318B70ABA0B29
:100E1000FE2E4108303E19000800003085003E30AB
:100E200084001F271F271F270230BA00003F303CD5
:100E3000031D1E2F20301A00BA0B162F0800083091
:100E4000BA00C101C035C10DF63041070318C10019
:100E50000318C00ABA0B222F4108303E19000800BF
:100E600043006F007000790072006900670068003D
:100E700074002000280043002900200032003000C8
:100E8000320030002D0032003000320032002000ED
:100E90006200790020004D002E00590061006D00B5
:0A0EA00061006D006F0074006F0028
:103F000003000000020004000000020003000000A3
:083F10000200000002000200A3
:020000040001F9
:02000E00840963
:02001000FB30C3
:00000001FF
